:100FA700EA600001010100000201010301010401DF
:100FB70001050101060101070101080101090101FC
:100FC7000A01010B00000C00000D00000E00000FCD
:100FD70000001000001100001200001300001400B0
:100FE7000015000016000017000018000019000087
:030FF700FAFAFA09
:10004900750B00750A00AE0AAF0BAC08AD09EDC31C
:100059009FEC9E401674FF120FFA75CF01780B744E
:100069000126F6500418E436F650DB2290006CE0C5
:10007900B4AA1A900790E0B43C13E5244523600D17
:10008900AE23AF24741EBE0004D39F50030201BCEB
:1000990090006AE4F0A3F075F809AE23AF24740761
:1000A9008E048F05FF12100AED4C7006743A900702
:1000B90090F0AE23AF247408BE001ED39F401A7E71
:1000C900017F08AC23AD241DBDFF011C12002E9039
:1000D9000068EEF0A3EFF0801FAE23AF247408127E
:1000E900103D8F048E057E017F08CDCCCD12002EE8
:1000F900900068EEF0A3EFF090006AE0FEA3E0FF45
:10010900740CD39F74019E50030201B7A2F9B35036
:10011900030201B4EF4E700375A38290006AE0FEFA
:10012900A3E0FF74016F4E700375A30090006AE0AD
:10013900FEA3E0FF74026F4E700BE52475F002A474
:10014900FDACF08DA390006AE0FEA3E0FF74036F9D
:100159004E700375A30090006AE0FEA3E0FF7403EC
:10016900BE00039F5017900068E0FCA3E0FDED2F4F
:10017900FFEC3EFE90008C121016E0F5A390006A89
:10018900E0FEA3E0FFEFB40B09EEB401057414120D
:100199000FFA90006AE0FEA3E0FFEFB40B07EEB49C
:1001A900010375F80D90006A12001E02010190000A
:1001B9006CE4F02290006AE4F0A3F075F809AE232C
:1001C900AF247408BE001ED39F401A7E017F08AC7D
:1001D90023AD241DBDFF011C12002E900068EEF016
:1001E900A3EFF0801FAE23AF24740812103D8F04D3
:1001F9008E057E017F08CDCCCD12002E900068EED1
:10020900F0A3EFF090006AE0FEA3E0FF7411D39F22
:1002190074019E500302031BA2F9B3500302031891
:10022900EF4E700375A3D290006AE0FEA3E0FF745D
:10023900016F4E700375A30090006AE0FEA3E0FF12
:1002490074026F4E700BE52475F002A4FDACF08DBD
:10025900A390006AE0FEA3E0FF74036F4E7003757C
:10026900A30090006AE0FEA3E0FF74046F4E7003E0
:1002790075A30090006AE0FEA3E0FF74056F4E705D
:100289000375A30090006AE0FEA3E0FF74066F4EB9
:10029900700375A30090006AE0FEA3E0FF74076F86
:1002A9004E700375A30090006AE0FEA3E0FF740896
:1002B9006F4E700375A30090006AE0FEA3E0FF741F
:1002C90008BE00039F501A900068E0FCA3E0FDED12
:1002D9002FFFEC3EFE900087121016E5A3F075A3E0
:1002E9000090006AE0FEA3E0FFEFB41009EEB4014C
:1002F900057414120FFA90006AE0FEA3E0FFEFB450
:100309001007EEB4010375F80D90006A12001E0281
:10031900020D22C203C2042290006CE0B4AB028039
:10032900030203DB90006AE4F0A3F075F80990007A
:100339006AE0FEA3E0FF7427BE0004D39F500302C6
:1003490003DBA2F9B350030203D8EF4E700375A380
:100359008290006AE0FEA3E0FF74016F4E7003759E
:10036900A30090006AE0FEA3E0FF74026F4E700BD9
:10037900E52475F002A4FDACF08DA390006AE0FEBF
:10038900A3E0FF74036F4E700375A30090006AE049
:10039900FEA3E0FF7403BE00039F50099000691299
:1003A9001016E0F5A390006AE0FEA3E0FF74266F43
:1003B9004E70057414120FFA90006AE0FEA3E0FF74
:1003C90074266F4E700375F80D90006A12001E02B4
:1003D90003372290006AE4F0A3F075F80990006AE7
:1003E900E0FEA3E0FF7427BE0004D39F500302047C
:1003F900E2A2F9B350030204DFEF4E700375A3D2F2
:1004090090006AE0FEA3E0FF74016F4E700375A3CC
:100419000090006AE0FEA3E0FF74026F4E700BE5E6
:100429002475F002A4FDACF08DA390006AE0FEA350
:10043900E0FF74036F4E700375A30090006AE0FE3D
:10044900A3E0FF74046F4E700375A30090006AE087
:10045900FEA3E0FF74056F4E700375A30090006A58
:10046900E0FEA3E0FF74066F4E700375A3009000D1
:100479006AE0FEA3E0FF74076F4E700375A3009056
:10048900006AE0FEA3E0FF74086F4E700375A300D5
:1004990090006AE0FEA3E0FF7408BE00039F500CC1
:1004A900900064121016E5A3F075A30090006AE0AD
:1004B900FEA3E0FF74266F4E70057414120FFA90B4
:1004C900006AE0FEA3E0FF74266F4E700375F80D15
:1004D90090006A12001E0203E62290006CE0B4ABA1
:1004E90002800302059D90006AE4F0A3F075F80903
:1004F90090006AE0FEA3E0FF7427BE0004D39F507A
:100509000302059DA2F9B3500302059AEF4E700349
:1005190075A38290006AE0FEA3E0FF74016F4E703C
:100529000375A30090006AE0FEA3E0FF74026F4E1A
:10053900700BE52475F002A4FDACF08DA390006A60
:10054900E0FEA3E0FF74036F4E700375A3009000F3
:100559006AE0FEA3E0FF7403BE00039F5009900008
:1005690069121016E0F5A390006AE0FEA3E0FF749B
:10057900266F4E70057414120FFA90006AE0FEA3FC
:10058900E0FF74266F4E700375F80D90006A120033
:100599001E0204F922C293C294C291C292C287C2B6
:1005A90090E5B554EFF5B5E5B554DFF5B5E5B554C6
:1005B900FBF5B52290008BE0FEA3E0FF900FA91296
:1005C9001016E493F59974506F4E700375330090CB
:1005D900008B12001E22C2AF75D904758F0175B741
:1005E900A575B7F17406900047F0758F00D2AF7505
:1005F900D94422C2AF75D904758F0375B7A575B7EC
:10060900F190F800E4F0758F00D2AF75D94422E576
:100619003464046006E59964FF60028031A20040F9
:1006290004D2008027E534600874E6253490008EF2
:10063900F0E533600874F0253390008EF0E534B4AA
:10064900010280FE753400753300C2008002C200C9
:10065900E534900E54F8282873753400E599B4FFF1
:1006690003753301E599B4FE03753302E599B4FDC9
:1006790003753303E599B4FC03753304E599B4FABA
:1006890003753305E599B4FB0675340112059EE53A
:1006990099B4F90675340412059E90008BE4F0A311
:1006A900F0D2990209D890008BE0FEA3E0FF9000F8
:1006B90090121016E599F090008B12001E90008B95
:1006C900E0FEA3E0FFEFB40106EEB40702800302E7
:1006D90007E0900790E0B43C0280030207D775FF5A
:1006E900A0C29C12031C90012EE090006DF09000B6
:1006F9009DE090006EF09000BDE090006FF09000DA
:10070900E6E0900070F0900092E0900071F09000A7
:10071900D8E0900072F09000F6E0900073F090003D
:10072900CAE0900074F09000E8E0900075F0900144
:1007390018E0900076F07400900077F07400900053
:1007490078F07400900079F075246375230074AB18
:1007590090006CF012032190006CE4F07509647547
:100769000800120049754701E547D39407502085D1
:10077900472475230074AA90006CF012007575095E
:10078900647508001200497847740126F650D97437
:100799003C900790F0754708E547D3940E502085A3
:1007A900472475230074AA90006CF012007575092E
:1007B900647508001200497847740126F650D9D2A9
:1007C9009C7599FB80FE7524C8752300D29C759988
:1007D900FF7534007533000209D80209D80209D817
:1007E90090008BE0FEA3E0FF900090121016E599AF
:1007F900F090008B12001E90008BE0FEA3E0FFEF4B
:10080900B40006EEB4010280030209D875FFA09076
:100819000058E0D394C7400B900058E0C394C8F542
:1008290035801A900058E0D39463400B900058E04B
:10083900C39464F5358006900058E0F535E53575C3
:10084900F002A4FFAEF08F47EF90009012102BEF4B
:10085900FCE0FDEC90009312102BEDFCE0FDEC2D7B
:10086900B5350280030209CA0FEF90009012102BD0
:10087900E547FFE0FCEF90009412102BECFFE0FC41
:10088900EFC39CB5350280030209CAE5479000927F
:1008990012102BE547FFE0FCEF90009512102BECAE
:1008A900FFE0FCEF2CB5350280030209CAE5479049
:1008B900009612102BE0C3953590006DF0E5479036
:1008C900009712102BE0C3953590006EF0E5479024
:1008D900009812102BE0C3953590006FF0E5479012
:1008E900009912102BE0C39535F524752300740087
:1008F900900070F074FF900071F0E54790009A1233
:10090900102BE0C39535900072F0E54790009B12DB
:10091900102BE0C39535900073F0E54790009C12C9
:10092900102BE0C39535900074F0E54790009D12B7
:10093900102BE0C39535900075F074AB90006CF006
:100949001204E3750964750800120049782312102E
:10095900451204E3750964750800120049782312E9
:1009690010451204E3750964750800120049AE23A5
:10097900AF24740412103D8E238F24900056E0900A
:10098900006DF0900057E090006EF0900058E090F4
:10099900006FF07437900070F01204E37509647504
:1009A9000800120049900047E493640660031205A9
:1009B900DF900062E0540260031205FC7599F9802A
:0F09C900FE7599FF75096475080012004980FEDC
:0F0E54000206620206AF0207E30207E60207E9A1
:1009D80022E533900E63F8282873020ADE90008B14
:1009E800E0FEA3E0FF900048121016E0F599900091
:1009F8008B12001E90008BE0FEA3E0FF741C6F4E6C
:100A08007003753300020ADE853F99020ADE900002
:100A18008BE0FEA3E0FF900090121016E0F599EF2E
:100A2800B40107EEB4070375330090008B12001E63
:070A3800020ADE90008CE0D1
:0F0E63000209E20209E5020A10020A16020A3B1E
:100A3F00900E75F8282873852899020AD3759900A6
:100A4F00020AD3853899807C853A998077853C99BD
:100A5F008072853E99806D85409980688541998027
:100A6F0063854299805E8543998059853D9980546D
:100A7F00759900804F759900804A7599008045904F
:100A8F00008EE0F599803D7599008038759900804A
:100A9F0033759900802E75990080297599008024EF
:100AAF00759900801F759900801A759900801575CA
:100ABF0099008010759900800B75990080067599C3
:040ACF00FC7533007F
:100E7500020A46020A4C020A52020A57020A5C0298
:100E85000A61020A66020A6B020A70020A75020A00
:100E95007A020A7F020A84020A89020A8E020A96E7
:100EA500020A9B020AA0020AA5020AAA020AAF02C6
:100EB5000AB4020AB9020ABE020AC3020AC8020A31
:010EC500CD5F
:0B0AD30090008B12001E80031205BD76
:030E7200020ADB96
:100ADE0022C2CF05462290F800E493640660089087
:100AEE000047E493B40602800280FE75840175A768
:100AFE000075FF8075EF0690006CE4F075C91075F7
:100B0E00A70F75A1C775A70075D90075CE0C75A76F
:100B1E000F75F1FE75F2FF75F30775F47875A4DAAB
:100B2E0075A5FF75A60775AE0075AFFF75D48175F7
:100B3E00D5FF75D6FF75D7FF75A70075A20175A1F4
:100B4E004775F80975D80075D90475DA0975DB098A
:100B5E0075E60875BC0175BE0475BD6C75BE07756E
:100B6E00BDA075BE0875BD0175BC0075BB1875BC02
:100B7E002075BA0875E88075D11375A70F75E10554
:100B8E0075E20075C74075B500C293C294C291C29A
:100B9E0092C287C290E5B554EFF5B5E5B554DFF5D1
:100BAE00B5C296C295C2A0C297C2A2C2A1E5B55463
:100BBE00BFF5B5E5B5547FF5B5E5B554FBF5B5759F
:100BCE009700759780740A120FFA7597C0E59754BF
:100BDE0020700280F8758F0275A700D2AF7598004D
:100BEE0075A90C75A70F75AB4375ADFB75AC1E756E
:100BFE00A700758912758E04758C00758A00C2A9BE
:100C0E00D28CD2ADC2CFD2CA75B62075D944753347
:100C1E0000753400C2997509C8750800120049752F
:100C2E00A70FE5FC900055F0E5FB900056F0E5FAB5
:100C3E00900057F0E5F9900058F075A70075470140
:100C4E00E547D3940750118547247523001201BD43
:100C5E007847740126F650E890F800E493B4066ED7
:100C6E0090F800E493900048F090F802E49390001E
:100C7E004BF090F803E49390004CF090F804E4935A
:100C8E0090004DF090F805E493900053F090F80624
:100C9E00E493900054F0900056E0900059F09000CC
:100CAE0057E090005AF0900058E090005BF090F8FA
:100CBE0007E493900062F0900062E0440A900062B4
:100CCE00F0900062E054FE900062F0020D5E740639
:100CDE00900048F0900047E493B40629752464759B
:100CEE0023001203DC7524C875230090006DE0907C
:100CFE000059F090006EE090005AF090006FE09076
:100D0E00005BF080127463900059F0746390005A87
:100D1E00F0746390005BF07524667523001203DC9B
:100D2E007524C875230090006DE090004BF0900084
:100D3E0074E090004CF090006EE090004DF0740066
:100D4E00900053F07401900054F07400900062F023
:100D5E007400900049F0740990004AF074009000FD
:100D6E004EF074F590004FF07404900050F0740043
:100D7E00900051F07401900052F0740090005CF0FD
:100D8E00740090005DF0740090005EF074009000AE
:100D9E005FF07400900060F07400900061F074FFDA
:100DAE00900063F0C20090008BE4F0A3F07400900A
:100DBE00009DF0752119752264900064740DF0A3E6
:100DCE0074ACF0754500743A900790F074FD90077E
:100DDE0091F074FA90008EF0753600752800752724
:100DEE0000753B007533007534007538007543008F
:100DFE00753A00753900753C00753D00753E0075FD
:100E0E004000754100754200900066E4F0A3F07555
:100E1E004400753F01D29CD2EC75CF01A298B3402D
:100E2E0005C298120618E5336006A299B3B34002C4
:100E3E008005C2991209D9E53464016005E534B420
:060E4E00040280D580D3F0
:09102B002582F5825002058322A2
:10103D00CFC39FFF50011E220806B60002180622DC
:0D001E00A3E004F07006121021E004F022AF
:10002E00EF8DF0A4F9A8F0EF8CF0A428F8EE8DF087
:06003E00A428FEE9FF22E8
:100FFA00600D782B021004007830D8FED5E0F82274
:0C100A00EEC0E07E00120EC6D0E0FE2218
:03002B00020003CD
:03000000021034B7
:0910340075814A75D000020AE43E
:0B101600E5822FF582E5833EF5832282
:100EC600BC000FBE0008ED8FF084FFADF022E4FEFB
:100ED600FF22BE000DEF60FE54F0606F20E70302B4
:100EE6000F7CEAC0E0EBC0E078017A0075F001EE15
:100EF60020E710EF25E0FFEE33FE0AC5F023C5F02C
:100F060030E7F0EA5407F9096A7A007B00600108C5
:100F1600C3EC9E40167004ED9F4010ED9FFDEC9EC5
:100F2600FCE5F0CA4ACA03F5F08005E5F003F5F0E2
:100F3600C3EE13FEEF13FFD9D77908CACBCAD8D0B0
:100F4600EAFEEBFFD0E0FBD0E0FA22EC8FF084FC67
:100F5600ED54F045F0C48FF084FEEDC454F045F036
:100F6600C48FF084FDEEC4FE54F02DFFEE540F3C0A
:100F7600FEADF07C0022790078008FF0EC7E082030
:100F8600E70DC3CD33CD33C933C9C833C8DEF084CA
:100F960049F9E5F08FF0BE00E6FD7C00E9FFE8FECA
:010FA6002228
:0A1021000582D58202158315822294
:10000300C0E0C0F0C083C082C0D075D000120ADF48
:0B001300D0D0D082D083D0F0D0E032FB
:00000001FF
